:02000000552881
:08000800FF00030E8301A000BC
:100010000A08A1008A010408A2000E288B1303130A
:1000200083120B1C2628061A1C28861A2128C43085
:10003000F0000130F1004828FF30F0000130F100FD
:100040004828FF30F0003C30F1004828700881005B
:100050007108F3070318F20A7208A83A031D36283C
:10006000BF307302031C3628F201F3000608043A7D
:100070008600061C4028A8309500971617124828BD
:10008000720895009712F31B97161712731B171619
:100090000B118B160B108B152208840021088A0087
:1000A000200E8300FF0E7F0E0900C430F0000130E7
:1000B000F100F201F301FF30A400FF30A500FF3092
:1000C0008520F3308320031383126400810183169B
:1000D000EF3081006400E8308100831270088100F5
:1000E0008316FF3092008312950197121712043085
:1000F00092000F3097000B118B160B108B158B177E
:10010000000080288228A5008728A4008A282508C6
:0A01100066000800240865000800DE
:02400E00623F0F
:00000001FF
